:03000000020100FA
:03000B0002022EC0
:120023000201A54144414D20452E203139393602010081
:20010000C200C201C20475220012012312014412012A90050412018212042E1203FF12019A
:2001200090212175B80275A8922275D000758780758922758DF3758BF3758921D28E759898
:2001400050D20322758CD8758AF0D28C22C0E075F00A842430F5993099FDC299E5F0243051
:20016000F5993099FDC29912016DD0E022C082C0833003FDC203900670858223858324D2D6
:2001800099223003FDC203858223858324D2992274007823900000F0A3D8FC782379257716
:2001A0000009D8FB222098030201F5C298C0E0E599B43F089005A212021C21EAB461022171
:2001C000EAB4650221EAB474081202E112030E21EAB473081202E11203AD21EAB464081299
:2001E00002E112036921EAB4760090065312021CD0E0D2A932C0E0C082C083C29985238249
:20020000852483740093600BF599A38582238583244115D203D083D082D0E03274009360A0
:200220000AF5993099FDC299A3411CD20322C28CB200758AF0758CD8D28CB2B5C0E0C0829F
:20024000C083E590B4FF12C2013004051203FFC2047522FF1203454173200104D2014173FB
:2002600030970D3004051203FFC20412027A41731202A6D083D082D0E032E590547FF521B6
:20028000B5220241A574009006CCC0E093B5210BD0E00412030E85212241A5D0E0B42202A8
:2002A00041A504418A2230040122D20412048874A01204E574507D239000001204E5120488
:2002C0008874A11204E51204F1120500F0A3DDF61204F11204CE223000FD2000FD3000FD7E
:2002E0002290065D12021C7B003098FDC298E599B40D02EB22F5993099FDC299943040E935
:20030000FC940A50E4EB75F00AA42CFB41E914F92448F8E6B4FF0B898275830074FFF00243
:20032000034412034512048874A01204E5E91204E5E92425F8E6F4F67583008982F0120488
:20034000E51204CE22C0E0C082C0837848E6B4FF0BE89448F5827583007400F008B85CED89
:20036000D083D082D0E022222214F99006A112021C3098FDC298E599B4611812048874A0D2
:200380001204E5E924501204E574FF1204E51204CE61ACB46EDB12048874A01204E5E924F4
:2003A000501204E574001204E51204CE2214F990067312021C3098FDC298E599B4691F74EA
:2003C0004829F87400F612048874A01204E5E924251204E574001204E51204CE61FEB4709A
:2003E000D4744829F874FFF612048874A01204E5E924251204E574FF1204E51204CE221283
:20040000048874A01204E574007D1490000078251204E512048874A11204E51204F1120548
:2004200000F6F008A3DDF41204F11204CE2212048874A01204E574257D1490000078481214
:2004400004E512048874A11204E51204F1120500F6F008A3DDF41204F11204CE2279147873
:2004600048C299E6B40005759949816F7599503099FDC29975990A3099FDC29975990D30F0
:2004800099FDC29908D9DC22D2B2D2B3000000000000C2B30000000000C2B220B2FD0022A9
:2004A00092B30000D2B230B2FD0000000000000000C2B200D2B300227400D2B230B2FD00A2
:2004C000A2B333A2B333C3C2B2006001D322C2B3000000D2B230B2FD0000000000D2B30022
:2004E00000000000227F08331204A0DFFA1204B8227F087400C0E01204B8D0E033DFF6225E
:20050000C391A022436F6E6E656374696F6E206120343830302062617564732C2038206213
:200520006974732C20706173206465207061726974652C20312073746F700A0D0A0D436514
:200540006E7472616C6520642765636C6169726167652041452D3133352E2020436F707958
:200560007772697465204144414D20452E20313939360A0D0A0D456E20617474656E6465AB
:2005800020646520636F6D6D616E64652E20283F203D2061696465290A0D41452D313335BD
:2005A0003E00416964652064657320636F6D6D616E6465206465206C612063656E74726157
:2005C0006C6520642765636C6169726167650A0D0A0D732020203D2020205479706520643E
:2005E0006520736F727469652028496E74657272757074657572202F20426F75746F6E2079
:20060000706F7573736F6972290A0D642020203D20202050726F6772616D6D6174696F6E55
:2006200020706F757220616C61726D650A0D742020203D2020204368616E6765206C27655C
:20064000746174206427756E6520736F727469650A0D000A0D41452D3133353E000A0D4396
:20066000616E616C206E2E3A2028312D333529000A0D000A0D69203D20496E7465727275B4
:20068000707465757220202020202070203D20626F75746F6E20506F7573736F69720A0D4B
:2006A000000A0D61203D204F4E20736920616C61726D202020202020206E203D204F4646D9
:2006C00020736920616C61726D0A0D00787472713C6C6A6665635C5A595655534E4D4B4791
:0F06E0003C3A393635332E2D2B271E1D1B171F85
:00000001FF
